:020000040800F2
:10000000700E002001010008272200084D1F000883
:100010002522000887010008293C00080000000094
:10002000000000000000000000000000EB260008B7
:10003000AD01000800000000AD25000805270008FC
:100040001B0100081B0100081B0100081B01000820
:10005000AF010008E92500081B0100081B0100088A
:100060001B0100081B0100081B0100081B01000800
:100070001B0100081B0100081B0100081B010008F0
:100080001B0100081B0100081B010008B53B00080C
:10009000C13B00081B0100081B0100081B010008F0
:1000A0001B0100081B0100081B0100081B010008C0
:1000B0001B0100081B0100081B0100081B010008B0
:1000C0001B0100081B0100081B0100081B010008A0
:1000D0003D260008592A00081B0100081B010008E2
:1000E0001B0100081B0100081B010008DFF80CD0F1
:1000F00000F02AF800480047993C0008700E0020E4
:100100000648804706480047FEE7FEE7FEE7FEE7B1
:10011000FEE7FEE7FEE7FEE7FEE7FEE791270008C1
:10012000ED00000840EA01039B0703D009E008C97D
:10013000121F08C0042AFAD203E011F8013B00F8AC
:10014000013B521EF9D27047064C074D06E0E068AD
:1001500040F0010394E8070098471034AC42F6D30E
:10016000FFF7C8FFC8410008E841000810B5142097
:1001700002F03CFA800705D10321BDE810401420AD
:1001800002F0B4BA10BDFEE70020704700207047AF
:100190000020704770B50C46054602F027FA20EAA9
:1001A00004012846BDE8704003F040BD704700F0F0
:1001B0008DB80000064A0021D16106490A6942F063
:1001C00002020A614861086940F040000861704716
:1001D0002801002000200240044B0022DA61044A7A
:1001E000136943F001031361018070472801002067
:1001F0000020024008490948096801600649091DB4
:1002000009684160044908310968816002490C317C
:100210000968C1607047000000FC00083A0800202F
:100220000E49C868C2060E4803D5C26942F00202F0
:10023000C261CA68520703D5C26942F00102C261B5
:10024000CA69D20707D0C26942F00402C261C86914
:1002500020F00100C8611420C860704700200240EF
:100260002801002070B5114C114E00F0F1F8304615
:10027000FFF7A0FF00F0AEF800F0EAF80025002339
:1002800031460220226800F0B1F8002331460220F6
:10029000226800F0ABF86D1CADB2241D361D042D94
:1002A000EDD3BDE8704000F095B800003A0800209A
:1002B00000FC000831B500F0C5F9044600F0C2F9B1
:1002C0000099001B8842F9D338BD70472DE9F041F1
:1002D0003E4DE8683E4CC0064FF0FF374FF0000639
:1002E00002D4E868400708D5D4F80880A760FFF773
:1002F00097FF404600F078F82670E868800653D5EE
:100300002020E8602078F8B1207801281DD02078DE
:10031000022833D06068401E60606068B0B3A06897
:10032000801CA060A06821696269090C41EA024151
:10033000120C21616261296921F0010129612169A1
:10034000626989B2FFF748FF2EE06068401E606076
:10035000606868B1A068FFF7B8FFA06800F580602A
:10036000A060296921F002012961FFF723FF1BE04A
:100370003846A7602670FFF7A8FF15E0286920F02F
:10038000040028610020FFF7A0FF0CE0FFE72078C1
:10039000032817D020780428A06815D0B0F10600F3
:1003A000FFF793FFA76026702078002808D12869FE
:1003B00020F007002861286920F4A05028612676E3
:1003C000BDE8F081A068EBE7801EE9E7002002406D
:1003D000280100200348016941F0800101610020EB
:1003E0007047000000200240704700002DE9F041F6
:1003F0000D46014614480024067E012E1AD0134FE4
:1004000001260676D7F810C04CF4A05CC7F810C0DF
:1004100085600261436101290ED0042302290FD0B7
:1004200005210170436091B22846FFF7D5FE2046B2
:10043000BDE8F0810220FBE7032101704660F2E78E
:10044000037002214160EEE72801002000200240F5
:1004500005480169090605D5044941600449416020
:1004600000207047012070470020024023016745AB
:10047000AB89EFCD2DE9F84FDFF890A100220AF10A
:10048000040B144601274FF00F090BF1040E00BFB7
:100490000B6807FA04F52B40AB4274D1DFF870C14A
:1004A0004E68A6EB0C0866452BD00DDC032E34D02D
:1004B00005DC36B3012E19D0022E2FD11BE0112EF0
:1004C00016D0122E2AD119E0B8F5881F19D006DCF3
:1004D000B8F5803F15D0B8F5801F1FD111E0B8F5F1
:1004E000001F0ED0B8F5041F18D10AE0CA6815E045
:1004F000CA68121D12E0CA6808320FE0CA680C32DE
:100500000CE08A682AB1012A4FF0080203D0456145
:1005100004E0042202E0056100E00022FF2B01D884
:10052000064601E000F104064FEA840501D9A5F171
:100530002005D6F800C009FA05F82CEA080C02FAE2
:1005400005F54CEA050CC6F800C04D68ED0057D51E
:10055000304DAE6946F00106AE61AD6924F0030688
:1005600005F0010500952C4D06EB050CDCF8085054
:10057000A6074FEA167809FA08F6B543274EB042A7
:1005800002D1002610E03BE0254EB04201D1012609
:100590000AE0244EB04201D1022605E0224EB042CC
:1005A00001D1032600E0042606FA08F62E43CCF813
:1005B00008604D68DAF80060ED03554601D51E432A
:1005C00000E09E432E604D68DBF80060AD035D46A1
:1005D00001D51E4300E09E432E604D68DEF80060AA
:1005E000ED02754601D51E4300E09E432E604D6826
:1005F000AD020E4D2E6801D51E4300E09E432E60D5
:10060000641C102CFFF444AFBDE8F88F00040140D7
:1006100000001110001002400000014000080140DD
:10062000000C014000100140001401400C04014086
:100630008068084000D0012070470AB1016170470E
:100640000904FBE70148006870470000040000202F
:1006500002480168491C0160704700000400002046
:10066000074810B5016841F010010160032000F057
:1006700097F8002000F006F800F016F8002010BDF2
:100680000020024010B5044600F05EFC4FF47A7181
:10069000B0FBF1F001F06FFB00222146501E00F08C
:1006A0005FF8002010BD0000254808B5816941F0C1
:1006B00001018161806900F001000090032000F0D9
:1006C0006FF8002211466FF00B0000F049F800228D
:1006D00011466FF00A0000F043F8002211466FF057
:1006E000090000F03DF800221146501F00F038F8D4
:1006F00000221146101F00F033F800221146901E10
:1007000000F02EF800221146501E00F029F80022B9
:100710001146042000F024F8042000F015F800220F
:100720001146052000F01CF8052000F00DF80548E2
:10073000416821F0E06141F00071416008BD0000B6
:10074000001002400000014000F01F020121914012
:100750004009800000F1E020C0F80011704700005F
:10076000F0B40E4B1B680C46C3F30223C3F107051C
:10077000042D00D90425191D072901D2002300E00A
:10078000DB1E012606FA05F1491E214099409E40D4
:10079000761E16403143F0BC01F047BD0CED00E081
:1007A000064900F0070208684FF6FF03184040EAC8
:1007B0000220034A10430860704700000CED00E07F
:1007C0000000FA0510B50C0605D501F07F0100EB1D
:1007D0004110283003E000EB411000F5027099B29F
:1007E00032B101228272C180190C0181002010BD3A
:1007F000002282728180F9E7704700EB4112D0F845
:100800001C04D26B02F0ADBB00EB4112D0F81C040B
:10081000D2F81C2202F0FABB10B504460A460B06B9
:1008200001F07F0004EB401101D5283101E001F512
:1008300002710870D009487094F8E803012809D0C3
:10084000012084F8E803206802F0D6FF002084F835
:10085000E80310BD022010BD70B50A460446090623
:1008600002F07F0003D504EB4011283103E004EBD4
:10087000421101F5027100258D700870D009487091
:1008800094F8E803012809D0012084F8E8032068DF
:1008900003F05AF884F8E853002070BD022070BDC0
:1008A00070B504460D460E0601F07F0004EB4011C2
:1008B00001D5283101E001F502710870E80948709E
:1008C0000A61CB7094F8E803012809D0012084F86C
:1008D000E803206802F060FE002084F8E80370BDA1
:1008E000022070BD70B504460E4601F07F0004EB97
:1008F000401101F5077100252CC101F81F5C01F8BA
:10090000200D94F8E80301280AD0012084F8E803B8
:100910007006206803F072F884F8E853002070BD78
:10092000022070BD70B50D460446090605F07F0033
:1009300003D504EB4011283103E004EB451101F528
:10094000027101228A700870E809487094F8E8037F
:10095000012807D084F8E823206803F02AF8680605
:1009600002D006E0022070BD04F57B71206802F021
:10097000E9FF002084F8E80370BD70B504460E4618
:1009800001F07F0004EB40113C3100252CC1012215
:1009900001F81F2C01F8200D94F8E803012809D074
:1009A00084F8E8237006206803F028F884F8E853F8
:1009B000002070BD022070BD10B50446006803F031
:1009C00005F9000402D5204601F03FFC206803F041
:1009D000FDF840050CD5206830F8441F21F48061F3
:1009E0000180204600F0ECF80021204600F0FDF8E0
:1009F000206803F0EBF8400405D5206830F8441F68
:100A000021F480410180206803F0E0F8800405D5DE
:100A1000206830F8441F21F400510180206803F061
:100A2000D5F8C00413D5206830F8401F21F0040128
:100A3000018021684FF43D40A1F84000204600F0BD
:100A4000CCF8206830F8441F21F4805101802068E0
:100A500003F0BCF800051AD5206830F8441F21F4D3
:100A600000610180206830F8401F41F008010180DA
:100A7000206830F8401F41F004010180206803F035
:100A8000A5F8C043C00402D5204600F0E3F8206872
:100A900003F09CF8800508D5206830F8441F21F445
:100AA00000710180204600F09CF8206803F08EF869
:100AB000C00505D5206830F8441F21F480710180FD
:100AC00010BD00002DE9F04186B004004FF0000594
:100AD00004D094F8E903002620B108E0012006B014
:100AE000BDE8F08184F8E863204600F04BF803206D
:100AF00084F8E903206802F01EFF04F110011422BB
:100B000088466846FFF70EFB94E80F0002F072FE7D
:100B10000021206803F06DF85FF0010704EB451039
:100B200080F8297000F8285F8581C67006614661EB
:100B30006D1C86610F2DF1D35FF0000004EB4011B6
:100B400081F8096281F80802888681F80B62C1F891
:100B50001862C1F81C62401CC1F820620F28EDD356
:100B6000142241466846FFF7DDFA94E80F0002F0D0
:100B7000D9FE84F8246084F8E973206802F0D0FE7E
:100B80000020ACE708B500680B49884212D10B4839
:100B9000C16941F40001C161C069002200F4000094
:100BA000009011461420FFF7DBFDBDE8084014203B
:100BB000FFF7CABD08BD0000005C00400010024005
:100BC00010B504460121D0F81C0402F0FFFAD4F855
:100BD0001C04BDE8104002F0C8BAD0F81C0402F0B2
:100BE000E3BAD0F81C0402F0E5BA10B5044690F858
:100BF000E80301280BD0012084F8E80384F82410CE
:100C0000206802F0F8FF002084F8E80310BD0220FD
:100C100010BDD0F81C2400F57B71104602F0E9BA33
:100C200010B5044690F8E803012810D0012084F89C
:100C3000E80301462046FFF7DFFD206802F06EFE64
:100C4000206802F0B0FF002084F8E80310BD022005
:100C500010BD000010B50446D0F81C0402F016FBCD
:100C6000A069002804D00348016841F00601016032
:100C700010BD000010ED00E02DE9F84305460078B6
:100C8000454CC00774D0E06940F08050E061E069F5
:100C9000424E00F080500090306840F48070306028
:100CA000FFF7D0FC074604E0FFF7CCFCC01B64282C
:100CB00033D83068C005F7D5206A10F4407051D0A1
:100CC000A98801F4407181424CD0206A0126310488
:100CD00091FAA1F2B2FA82F29300314A20F4407004
:100CE0001344C3F8006491FAA1F1B1FA81F102EB67
:100CF00081010023C1F800342062C00732D0FFF721
:100D0000A1FC074641F288394FF0020808E000BF15
:100D1000FFF798FCC11B494502D90320BDE8F883C1
:100D200098FAA8F1B1FA81F141F040014046B6EBE2
:100D3000511F01D121680BE090FAA0F1B1FA81F1C5
:100D400041F04001B0EB511F01D1216A00E0616A1E
:100D500098FAA8F0B0FA80F000F01F0206FA02F04C
:100D60000142D5D0206A696820F4407008432062AF
:100D70002878800705D56068A96820F440400843BA
:100D800060602878C00605D56068E96820F48000B6
:100D9000084360600020C1E700100240007000407E
:100DA00000004242704700002DE9F047DFF87081F3
:100DB00005460E46D8F8000000F00700B0420CD2FD
:100DC000D8F8001021F007013143C8F80010D8F816
:100DD000000000F00700B04277D12878514C80071E
:100DE00005D56068A96820F0F000084360602878A5
:100DF000C00759D06968012001290DD0022929D0E6
:100E00005FF0020393FAA3F2B2FA82F242F02002F8
:100E1000520904D0226803E04FF40033F2E7626A1B
:100E200093FAA3F3B3FA83F303F01F03984002424B
:100E30004BD0606820F0030008436060FFF702FCBD
:100E40006968074641F2883001290DD002298146A0
:100E500017D025E04FF00073D4E700BFFFF7F2FB97
:100E6000C11B494501D918E081466068C0F3810083
:100E70000128F3D118E000BFFFF7E4FBC11B49458F
:100E80000BD86068C0F381000228F5D10CE000BFE8
:100E9000FFF7D8FBC11B494502D90320BDE8F08705
:100EA000606810F00C0FF3D1D8F80010404601F044
:100EB0000701B1420BD9016821F0070131430160FC
:100EC000006800F00700B04201D00120E6E7287872
:100ED000400705D56068E96820F4E0600843606079
:100EE0002878000706D56068296920F4605040EA38
:100EF000C100606000F05EF86168F02292FAA2F230
:100F000001F0F001B2FA82F2D140074A515CC840C8
:100F1000064908600020FFF7B5FB0020BEE700008F
:100F20000020024000100240B041000820010020D3
:100F30000120C10491FAA1F1024AB1FA81F142F80B
:100F400021007047000042420148006870470000DD
:100F50002001002008480949006849684FF4E06210
:100F600092FAA2F201F4E061B2FA82F2D140044AAC
:100F7000515CC84070470000200100200010024072
:100F8000C041000808480949006849684FF46052A8
:100F900092FAA2F201F46051B2FA82F2D140044A0C
:100FA000515CC84070470000200100200010024042
:100FB000C041000810B519A385B00FCB8DE80F0014
:100FC0001AA01B4B006804905A681A4802F00C01E2
:100FD00004291DD008291BD14FF4701494FAA4F4ED
:100FE00002F47011B4FA84F4E140D2031DF8011048
:100FF00010D55A684FF4003393FAA3F302F4003289
:10100000B3FA83F3DA4004AB9A5CB0FBF2F04843E6
:1010100005B010BD08484843FAE700000203040584
:10102000060708090A0B0C0D0E0F10100102000034
:101030000010024000127A0000093D0010B5044C77
:10104000A068000603D5FFF7ADFE8020A07210BD9A
:10105000001002402DE9F84F04460078F74DC00714
:101060004FF0010625D068687704C0F3810001289D
:1010700007D06868C0F3810002281BD16868C003EC
:1010800018D597FAA7F0B0FA80F040F02000400998
:1010900001D0286800E0686A97FAA7F1B1FA81F1F7
:1010A00001F01F0106FA01F108425ED060680028D5
:1010B0007CD05AE06068B0F5803F0BD010B1B0F53D
:1010C000A02F11D0286820F480302860286820F4F0
:1010D000802002E0286840F480302860606828B3EF
:1010E000FFF7B0FA80460BE0286840F480202860C3
:1010F000F0E700BFFFF7A6FAA0EB0800642871D85C
:1011000097FAA7F0B0FA80F040F02000400901D033
:10111000286800E0686A97FAA7F1B1FA81F101F056
:101120001F0106FA01F10842E4D01EE0FFF78AFA37
:10113000804605E0FFF786FAA0EB08006428DED8B9
:1011400097FAA7F0B0FA80F040F02000400901D0F3
:10115000286800E0686A97FAA7F1B1FA81F101F016
:101160001F0106FA01F10842E4D12078DFF8D082AD
:1011700080074FF000094FF002075BD568684FF019
:10118000F80B10F00C0F07D06868C0F3810002283C
:101190001CD16868C00319D497FAA7F0B0FA80F0A0
:1011A00040F02000400902D0286801E08BE0686A26
:1011B00097FAA7F1B1FA81F101F01F0106FA01F1E6
:1011C00008422CD0206901287DD128E0206990B305
:1011D00096FAA6F0B0FA80F048F82060FFF732FAED
:1011E000824607E011E100BFFFF72CFAA0EB0A00EE
:1011F000022884D897FAA7F0B0FA80F040F02000D7
:10120000400901D0286800E0686A97FAA7F1B1FAAE
:1012100081F101F01F0106FA01F10842E4D02868CB
:101220009BFAABF26169B2FA82F220F0F8009140C9
:101230000843286025E0FFE796FAA6F1B1FA81F1AC
:1012400048F82190FFF7FEF9824605E0FFF7FAF92A
:10125000A0EB0A000228CCD897FAA7F0B0FA80F0E9
:1012600040F02000400901D0286800E0686A97FA41
:10127000A7F1B1FA81F101F01F0106FA01F108426C
:10128000E4D1207800076ED5A069B8B396FAA6F02D
:10129000B0FA80F008EB8000C0F88064FFF7D2F964
:1012A000824605E0FFF7CEF9A0EB0A000228A0D89D
:1012B00097FAA7F0B0FA80F040F06000B6EB501F4C
:1012C00002D128680CE062E197FAA7F0B0FA80F04A
:1012D00040F06000B7EB501F01D1286A00E0686A57
:1012E00097FAA7F1B1FA81F101F01F0106FA01F2B4
:1012F0001042D7D00120FEF7DDFF34E0FFE796FA79
:10130000A6F1B1FA81F108EB8101C1F88094FFF7F1
:1013100099F9824606E000BFFFF794F9A0EB0A00B6
:10132000022872D897FAA7F0B0FA80F040F0600077
:10133000B6EB501F01D128680BE097FAA7F0B0FA7E
:1013400080F040F06000B7EB501F01D1286A00E048
:10135000686A97FAA7F1B1FA81F101F01F0106FA64
:1013600001F21042D8D12078400765D5E86940F0F5
:101370008050E861E869DFF8CCB000F08050009060
:10138000DBF8001041F48071CBF80010FFF75AF938
:10139000824605E0FFF756F9A0EB0A00642834D82E
:1013A000DBF80000C005F5D5E06801280AD008B1D7
:1013B000052813D0286A20F001002862286A20F04E
:1013C000040002E0286A40F001002862E06841F26F
:1013D000883B90B3FFF736F982460BE0286A40F06D
:1013E00004002862EEE700BFFFF72CF9A0EB0A012A
:1013F00059450AD897FAA7F0B0FA80F040F04000BB
:10140000B6EB501F02D128680CE0A3E097FAA7F0D2
:10141000B0FA80F040F04000B7EB501F01D1286ACD
:1014200000E0686A97FAA7F1B1FA81F101F01F02B2
:1014300006FA02F10842D7D031E005E00010024080
:101440000000424200700040FFF7FCF8824605E0D1
:10145000FFF7F8F8A0EB0A0159457BD897FAA7F0F7
:10146000B0FA80F040F04000B6EB501F01D1286880
:101470000BE097FAA7F0B0FA80F040F04000B7EB2D
:10148000501F01D1286A00E0686A97FAA7F1B1FA03
:1014900081F101F01F0206FA02F10842D8D1E06999
:1014A00080B36968C1F38101022970D04FF0807167
:1014B0004F000228484609D091FAA1F1B1FA81F112
:1014C00048F82100FFF7BEF8044669E08A4691FA21
:1014D000A1F1B1FA81F1C14648F82100FFF7B2F855
:1014E000804605E0FFF7AEF8A0EB0800022854D8CC
:1014F00097FAA7F0B0FA80F040F02000400902D03F
:10150000286801E061E0686A97FAA7F1B1FA81F111
:1015100001F01F0106FA01F10842E3D1206AB0F59B
:10152000803F05D16868A16820F4003008436860F6
:10153000D4E908010843696821F47411084368601C
:101540009AFAAAF0B0FA80F049F82060FFF77AF82A
:10155000044606E021E000BFFFF774F8001B0228F4
:101560001BD897FAA7F0B0FA80F040F020004009AD
:1015700001D0286800E0686A97FAA7F1B1FA81F112
:1015800001F01F0106FA01F10842E5D01DE01EE05E
:10159000FFF758F8001B022802D90320BDE8F88F96
:1015A00097FAA7F0B0FA80F040F02000400901D08F
:1015B000286800E0686A97FAA7F1B1FA81F101F0B2
:1015C0001F0106FA01F10842E2D10020E6E70120FE
:1015D000E4E7704708B501684A68D243520609D467
:1015E0008A68D243D20705D18A68D243520601D510
:1015F000816C08E04A68D243120608D48A68D24354
:10160000920704D4C16C01B05DF804EB08474A6846
:10161000D243920635D48A68D243D20606D4426DAC
:1016200042F0020242656FF010028A6001688A6827
:10163000D243920609D4426D42F0010242658A68A3
:101640000A6822F040020A60009201688A68D24368
:1016500052060AD490F85120122A06D0426D42F068
:1016600004024265CA688A680092426D002A08D066
:101670004A6822F0E0024A60012180F85110FFF729
:10168000A8FF08BD10B5040003D094F8510010B1B4
:1016900004E0012010BD204600F038F8022084F854
:1016A00051002068016821F040010160D4E9010186
:1016B0000843D4E903121143084361690843218BAD
:1016C00001F400710843E1690843216A0843A16AF3
:1016D000084321680860A069042101EA1040616A9A
:1016E0000843216848602168E06A08612068C16990
:1016F00021F40061C1610449002008706065012087
:1017000084F85100002010BD0000002010B50068D2
:10171000164986B0884226D11548C16941F48041F6
:10172000C161C069134C00F4804004904FF4204024
:101730000090022001900320039069462046FEF7A6
:1017400099FE00214FF48040CDE9000102916946E5
:101750002046FEF78FFE002211462420FFF700F8F6
:101760002420FEF7F1FF06B010BD00000038004055
:1017700000100240000C01402DE9F84F00259A4668
:101780000446ADF8005090F8510001287ED1E9B32D
:10179000E2B394F85000012878D0012684F8506014
:1017A000222084F851006565A163A287E287A564C1
:1017B000E5642563A586E586A0684FF400494845A1
:1017C00004D12068036823F480430360A06A4FF4C7
:1017D0000057B84209D12068036823F4005303601E
:1017E0002068036843F40053036060684FF4827814
:1017F000404501D1A06878B120680168490603D44A
:10180000016841F040010160E06800E001E0E8B1FA
:1018100031E00120BDE8F88F84F8505013460A46A5
:101820002046CDF800A000F040F9F3E7534600222F
:101830000121204600F00AFF48BB2068C168A06B68
:10184000421CA2630170E08F401EE087E08F0128F8
:10185000ECD813E0534600220121204600F0F6FEAA
:10186000A8B92068C068A16B0880A06B801CA06329
:10187000E08F401EE087E08F0128EBD8A06AB842D5
:1018800007D12068016841F4805101E068E007E079
:101890000160534600220121204600F0D7FE08B126
:1018A0000320B7E7E0680028206817D0C068A16B64
:1018B0000880A06B801CA063E08F401EE087A06AB8
:1018C000B84217D1534600220121204600F0BEFE47
:1018D00050B1606D40F002006065E1E7C168A06B47
:1018E000421CA2630170E7E72068C068ADF8000001
:1018F000BDF80000606840450AD1A068484502D0A4
:10190000B0F5806F04D12068016821F040010160CA
:1019100084F85160A06AB8420DD120688068C04345
:10192000C00608D4204600F08FFE012807D02168A9
:101930006FF01000886084F8505000206AE7606DF6
:1019400040F0020060652068016821F400510160E8
:101950002068016841F40051016084F8505058E754
:10196000022057E72DE9F843044690F851009846C5
:10197000012870D139B332B394F8500001286AD0ED
:10198000012684F85060122084F851000025656516
:101990002163A286E286E564A564A563A587E58741
:1019A000A06A7703B84209D12068016821F4005188
:1019B00001602068016841F400510160A068B0F541
:1019C000004F03D007E00120BDE8F88320680168DC
:1019D00041F48041016020680168490603D4016830
:1019E00041F040010160E0680028606804D0D8B18F
:1019F000E08E012818D021E010B1E08E012808D136
:101A0000206B411C216321680078C860E08E401E75
:101A1000E0860004000C1FD043460022022120462D
:101A200000F014FEA8B9EBE7206B21680088C860BD
:101A3000206B801C2063E08E401EE0860004000CBA
:101A40000AD0434600220221204600F0FFFD002874
:101A5000EAD00320B8E726E0A06AB84204D12068A3
:101A6000016841F480510160434600220221204672
:101A700000F0ECFD30B9434601228021204600F001
:101A8000E5FD20B1606D40F010006065E1E7A06801
:101A900018B92068C1688068009084F8516084F8A3
:101AA0005050002090E702208EE72DE9F8430025F2
:101AB000DDF820800446ADF8005090F85100012870
:101AC00003D094F8510022287DD169B162B15BB195
:101AD00094F85000012876D0012684F8506094F8DC
:101AE0005100012803D005E00120BDE8F883322031
:101AF00084F851006565A263A387E3872163A38609
:101B0000E386A564E564A06A4FF40057B84209D1A2
:101B10002068016821F4005101602068016841F4E7
:101B20000051016020680168490603D4016841F052
:101B300040010160E0684FF48271B0F5006F6068A9
:101B400007D0002867D088426ED1E08E012862D08D
:101B50006AE020B188420CD1E08E012809D1206BC7
:101B600021680088C860206B801C2063E08E401EC6
:101B7000E086E08E80B9A06AB84244D1206801684E
:101B800041F4805101603EE02068C068A16B08808C
:101B9000A06B801CA0639EE04346002202212046E9
:101BA00000F054FD002874D1206B21680088C860C3
:101BB000206B801C2063E08E401E0004000CE08639
:101BC00009D1A06A00E0C7E0B84204D120680168EA
:101BD00041F480510160434600220121204600F07B
:101BE00035FD00286FD12068C068A16B0880A06B0C
:101BF000801CA063E08F401EE087E08E0028CBD1E0
:101C0000606800286AD1434600220121204600F086
:101C10001DFDF0BBB8E7206B411C216321680078F3
:101C2000C860E08E401EE086E08E98B9A06AB84297
:101C300004D12068016841F48051016043460022CC
:101C40000121204600F002FD18BB2068C068A16B8E
:101C5000087040E0434600220221204600F0F6FCD6
:101C6000B8B9206B411C216321680078C860E08E00
:101C7000401E0004000CE08607D1A06AB84204D1DF
:101C80002068016841F4805101600022434601212F
:101C900000E018E0204600F0D9FCA0B92068C16837
:101CA000A06B421CA2630170E08F401EE087E08EB3
:101CB0000028CFD1606888B9434600220121204620
:101CC00000F0C4FC08B103200FE72068C168A06BD6
:101CD000421CA2630170E08F401EE087A06AB842F8
:101CE00010D1434600220121204600F0AFFC18B17C
:101CF000606D40F002000FE02068C068ADF80000A1
:101D0000BDF80000434601228021204600F09EFCE1
:101D100020B1606D40F010006065D4E784F8516038
:101D2000A06AB84214D120688168C943C9060FD49B
:101D3000616D41F002016165016821F400510160AB
:101D40002068016841F40051016084F85050CBE6EE
:101D500084F850500020C8E60220C6E64FF0E0218B
:101D60000428086903D020F004000861704740F09F
:101D70000400FAE7704710B5401EB0F1807F01D330
:101D8000012010BD4FF0E02460610F21601700F0CA
:101D90004CFA0020A06107202061002010BD10B582
:101DA000FFF7E8FF10BD704738B5044600680168CA
:101DB000C26811F0010F02F4807204D01AB1E16B15
:101DC00041F00101E1630168C1F34002416901F0A2
:101DD000010122B119B1E26B42F00402E263026830
:101DE000C2F3800222B119B1E26B42F00202E26357
:101DF0000268C2F3C00222B119B1E16B41F00801DF
:101E0000E1630168C068C1F3401100F0200019B11E
:101E100010B1204600F0E0FC20680168C068C1F302
:101E2000C01100F0800019B110B1204600F0E0FDB3
:101E300021680868CA68C0F3801002F040020125DA
:101E400070B16AB1CA68204622F04002CA6094F8B4
:101E50003910322911D080F8395000BF00F075F8E0
:101E6000E06B002808D0206801684068009084F882
:101E700039502046FFF797FF38BD222180F83910EE
:101E8000ECE770B5040004D094F83900002510B1D7
:101E900006E0012070BD84F83850204600F020F89C
:101EA000022084F839002068C16821F40051C16023
:101EB000204600F0E5FC2068016921F490410161B1
:101EC0002068416921F02A0141612068C16841F41C
:101ED0000051C160E563012084F83900002070BD25
:101EE00010B50068154986B0884225D1144881692B
:101EF00041F4804181618069124C00F4804004907B
:101F00004FF4007000900220019003200390694676
:101F10002046FEF7AFFA00212015CDE9000102911D
:101F200069462046FEF7A6FA002211462520FEF754
:101F300017FC2520FEF708FC06B010BD0038014054
:101F4000001002400008014070477047FEE77CB572
:101F50000446002529460D2001F068FE93202070DC
:101F60002020607001A823460090022219460C2010
:101F700000F024F8010009D1225C401C5540C0B299
:101F80000428F9D3205CA84200D0022108467CBD79
:101F90007CB50C46054607210D2001F047FE257053
:101FA00001A823460090012219460C2000F006F8F3
:101FB00010B90199102900D002207CBD2DE9FF5FE6
:101FC00000270226DDF838A015468B468146B84624
:101FD0000C2805D0B9F10E0F05D11227102001E011
:101FE00077273020804647F08001022001F01EFE56
:101FF00080210420FEF7CEF880210A2000F076FB35
:102000000021012001F012FE002405E01BF804105D
:10201000092001F00BFE641CAC42F7D349460120B5
:1020200001F004FEB9F10C0F03D180210D2000F066
:102030005DFB4FF4FA65042000F0D8FA04466D1EEB
:1020400004D0E00702D114EA080FF4D080210D205B
:10205000FEF7A0F835B1062000F0C8FA10F01B0F0B
:1020600004D0022604B03046BDE8F09F00263C4074
:10207000E00700D00126B9F10C0FF3D10A2000F0DF
:10208000B5FA04460C2000F0B1FA10F007004FEA50
:10209000C40101D008390144CAF8001024B1102C41
:1020A00004D91024002503E00124FBE7002507E004
:1020B000092000F09BFA03994855034948556D1CC7
:1020C000A542F5D3CEE70000200800202DE9F0431B
:1020D000324885B0816941F010018161816901F068
:1020E00010010491816941F020018161816901F051
:1020F00020010491816941F004018161816901F04D
:1021000004010491816941F0080181618069244FD3
:1021100000F008004FF40054049000222146384695
:10212000FEF78BFADFF87C80002204214046FEF7A0
:1021300084FADFF874906610002231464846FEF7B4
:102140007CFA0125CDE9004502246946384603940E
:10215000FEF790F90420CDE9000569460394404656
:10216000FEF788F9CDE90065694648460394FEF715
:1021700081F9E0010025CDE9000569460294484651
:10218000FEF778F92002CDE9000569460294484639
:10219000FEF770F905B0BDE8F083000000100240C2
:1021A0000010014000080140000C01400E4810B52D
:1021B0000C4901604FF48271416000218160C1606F
:1021C0004FF400720161C0E905121822C0E907212D
:1021D000416281620A21C162FFF754FA002800D0EF
:1021E000FEE710BD003800408807002010B500222F
:1021F0000849094800F080FE0849074801F073F8D3
:102200000749054800F0A1FCBDE81040024801F074
:10221000B7B80000DC0000204C0800200C000020B3
:10222000CC000020FEE7FEF709BF0907090E0028D1
:1022300006DA00F00F0000F1E02080F8141D70476E
:1022400000F1E02080F8001470472DE9FC5F4FF0AA
:1022500000080446ADF80480ADF8008048F60F7B16
:102260004FF002094FF4806692E1BDF8041011F0BE
:102270000F072BD030F82710ADF80010BDF8001074
:10228000090478D530F8272040F68F710A4020F8ED
:10229000272004EB471595F8120205F50275002872
:1022A000206869D0297830F8212052047DD5B0F813
:1022B000503009EBC101194406EB4101415AC1F309
:1022C00009015FEA010A71D0EA88D0E0BDF8041084
:1022D000C9062AD4018801EA0B010180206804F1B3
:1022E0002805B0F850202B7809EBC301114406EB08
:1022F0004101405AC0F309006064E16B0844E063A7
:1023000000212046FEF779FA94F824000028ABD08B
:10231000A8690028A8D194F82400216840F0800022
:10232000A1F84C0084F8248032E1018804F502759C
:10233000ADF80010BDF8001009051ED5B0F85030FA
:102340002978062202EBC101194406EB4101405AEB
:1023500004F57B71C0F30903EB61AA88206801F0E2
:1023600039FC2068018840F68F72114001802046B8
:10237000FEF74FFC0CE1A0E055E0BDF800100904A9
:10238000D2D5028840F68F710A4002802068B0F8EA
:1023900050302978062202EBC101194406EB4101B5
:1023A000405A83059B0DEB6101E051E063E008D0EA
:1023B000AA886969206801F00DFCE9696869084428
:1023C000686100212046FEF71FFA2068B0F850101F
:1023D000891D06EB4101014428693E280CD9C0F350
:1023E0004F12C00601D1521E92B24FF6FF7000EAA2
:1023F000822040F4004009E0C0F34F02C00701D042
:10240000521C92B24FF6FF7000EA822008602168E9
:1024100008884BF68F72104080F4405048F28002DA
:1024200010430880B4E0B0F850202B78062101EB6F
:10243000C301114406EB4101415AC1F309015FEAAE
:10244000010A24D0AA885346696901F0C3FB1EE043
:10245000B0F85020062303EBC101114406EB410103
:10246000415AC1F309015FEA010A04D02A8953469F
:10247000696901F0AFFB2978206830F8213048F60F
:102480008F72134048F2C002134320F82130E969EB
:1024900001EB0A00E861696901EB0A026A61AB6954
:1024A00013B12869504504D929782046FEF7ACF9C4
:1024B00003E029782046FEF715FABDF80000000673
:1024C00066D5206804EB471530F8271001EA0B01A8
:1024D00020F8271095F8320028350028206812D0FF
:1024E000297830F82120B0F8503052061ED509EB7B
:1024F000C101194406EB4101405A83059B0DEB6174
:1025000024D0EA881EE0B0F850302A7809EBC201E6
:10251000194406EB4101405A83059B0DEB6121D024
:10252000AA886969206801F06CFB1BE0062202EBB7
:10253000C101194406EB4101405A83059B0DEB6133
:1025400004D02A896969206801F05BFB297820683A
:1025500030F8212048F68F731A404CF280031A435A
:1025600020F821202068B0F850202B7809EBC30117
:10257000114406EB4101405AC0F30900E861696962
:102580000A186A612978AB69204663B1FEF7F5F94C
:102590002068B0F84410ADF8041009043FF565AEAA
:1025A0000020BDE8FC9FFEF728F9F1E7704710B561
:1025B0008D212A2001F03AFB3E212B2001F036FB31
:1025C0001E212C2001F032FB00212D2001F02EFBDA
:1025D0004021152001F02AFB3D21112001F026FBAE
:1025E000BDE81040FDF7C2BD704700007CB57E21FC
:1025F00001EA400040F080000E4D8DF800004FF4DD
:102600008054002221462846FEF717F86423012251
:1026100069460948FFF7A6F96423012201A9064883
:10262000FFF7AAF8012221462846FEF706F89DF892
:1026300004007CBD000C0140880700200148FEF723
:10264000C9BF000088070020012070472DE9F0472E
:102650001D4690460E460446FDF7F4FF07465FEA26
:1026600008004FF000084FF4005A4FF0010926D03F
:1026700034E0681C23D025B1FDF7E4FFC01BA8425D
:102680001DD92068416821F0E0014160206801689F
:1026900021F040010160A06A504509D1206801681D
:1026A00021F4005101602068016841F4005101608B
:1026B00084F8519084F850800320BDE8F0872068AA
:1026C000806836EA0000D4D10DE0681C06D0002DE9
:1026D000D7D0FDF7B7FFC01BA842D2D820688068CA
:1026E00036EA0000F1D00020E7E7704770B50C46ED
:1026F0000546FFF77BFF40EA04012846BDE870402D
:1027000001F094BA10B5FDF7A3FFBDE81040FFF744
:1027100046BB30B593B001210804CDE90010002478
:10272000029402250491CDE9075000010990684602
:10273000FEF790FC00B1FEE70F20CDE90A054FF44B
:102740008060CDE90C4001210AA80E94FEF72CFB15
:1027500000B1FEE710200F90800412900FA8FEF742
:102760008BFA00B1FEE7FEF7E3FBFEF7EDFB4FF45B
:102770007A71B0FBF1F0FFF7FEFA0420FFF7EEFAF2
:1027800000221146501EFDF7EBFF13B030BD0000D4
:102790000D48016841F00101016041680B4A114098
:1027A000416001680A4A11400160016821F48021FA
:1027B0000160416821F4FE0141604FF41F01816016
:1027C0000449C00308607047001002400000FFF891
:1027D000FFFFF6FE08ED00E010B590F83910222951
:1027E00003D0322901D0022010BD8168B1F5805F8D
:1027F00011D00169002901681FD0496801F07F03E9
:10280000816A4A1C82620B70C18D491E0904090C41
:10281000C18518D030E00269816A002A02685268D6
:1028200005D0D2B20A80816A491C8162ECE7C2F30A
:1028300008020A80816A891CF7E74A68816A4B1C92
:1028400083620A70E0E70168CA6822F02002CA6069
:1028500090F83910322911D00168CA6822F48072C8
:10286000CA6001684A6922F001024A615FF0010111
:1028700080F83910FFF768FB002010BD1221F7E740
:102880002DE9F041044600680169E26821F44051F5
:10289000114301612169A068084361690843216807
:1028A000CA6841F20C639A430243CA6020684169D6
:1028B000A26921F44071114341614C4920686425AB
:1028C000322688423CD1FEF75DFB00EBC00101EBF4
:1028D000001061688900B0FBF1F7FEF753FB00EBD5
:1028E000C00101EB00106168B0468900B0FBF1F057
:1028F000B0FBF5F06FF01801484307EB800106EBE1
:102900000110B0FBF5F000F0F006FEF73BFB00EB2A
:10291000C00101EB001061688900B0FBF1F0B0FB71
:10292000F5F006EB0016FEF72DFB00EBC00101EB06
:10293000001061688900B0FBF1F7FEF723FB3BE074
:10294000FEF708FB00EBC00101EB00106168890095
:10295000B0FBF1F7FEF7FEFA00EBC00101EB00104F
:102960006168B0468900B0FBF1F0B0FBF5F06FF0A4
:102970001801484307EB800106EB0110B0FBF5F0AE
:1029800000F0F006FEF7E6FA00EBC00101EB0010E4
:1029900061688900B0FBF1F0B0FBF5F006EB0016C2
:1029A000FEF7D8FA00EBC00101EB00106168890066
:1029B000B0FBF1F7FEF7CEFA00EBC00101EB00101F
:1029C00061688900B0FBF1F0B0FBF5F06FF0180121
:1029D000484307EB800108EB0110B0FBF5F02168DC
:1029E00000F00F0030448860BDE8F08100380140FD
:1029F00090F83910122903D0322901D002207047F3
:102A00008168B1F5805F016A0BD04A1C02620268DE
:102A100009785160C18C491E0904090CC1840ED08B
:102A200017E009880268C1F30801516001690029B3
:102A3000016A02D0491C0162ECE7891CFBE70168CE
:102A4000CA6822F08002CA600068C16841F0400193
:102A5000C1600020704700000148FFF7A5B90000E1
:102A6000E0070020D0F818020021017608467047E0
:102A700070B50546D0F81842D5F81C226178D268A6
:102A800020789047082322460121284600F05DFB6C
:102A9000002070BD10B50446812100F052FA0121DA
:102AA000204600F04EFAD4F8180250B1D4F81C02B7
:102AB00004F5067480688047206800F067FD0020F8
:102AC0002060002010BD10B5D0F8184261690129BE
:102AD00008D1D0F81C0223786178C2681846904764
:102AE00000206061002010BD29210180004870474E
:102AF000480000200A210180004870478000002023
:102B000070B50646002502230322812100F00AFB4E
:102B1000022303220121304600F004FB1C2000F0B8
:102B200037FDC6F8180270B1044600202076D6F8AA
:102B30001C0240688047082322460121304600F0ED
:102B400004FB284670BD0125FBE702460220002950
:102B500002D00020C2F81C12704710B5134690F83E
:102B6000FC41D0F81822032C07D1147E2CB9012483
:102B700014760A46812100F092FB002010BD00006F
:102B800070B500220D78D0F81832144615F06005A3
:102B900026D0202D4CD14A78921E0A2A1CD2DFE87A
:102BA00002F010081B1B1B1B1B140C058878986077
:102BB0003EE0012203F1080131E04888000AD860B4
:102BC00036E0012203F10C0129E001225A618A79E1
:102BD000194600F053F82BE000F045F8022070BDD4
:102BE0004D78062D04D00A2D1CD00B2D20D11DE0D0
:102BF0004B882225B5EB132F07D1CA883F2A00D96D
:102C00003F22D0F81C120C6808E02125B5EB132FE9
:102C100004D1CA88074C092A00D90922214600F0AC
:102C200047F805E0012203F11001F8E78878186100
:102C3000002070BD7400002010B5D0F81422526836
:102C40009047002010BD134610B50A46002100F041
:102C50007CFA002010BD134610B50A46002100F092
:102C60001EFB002010BD10B50446802100F0EEFAD6
:102C70002046BDE81040002100F0E8BA10B503235B
:102C8000C0F80821C0F8F431C0F80C2113460A46F8
:102C9000002100F05AFA002010BD10B505210023D4
:102CA000C0F8F4111A46194600F04FFA002010BD82
:102CB00010B502238261C0F8F431C26113460A469E
:102CC000002100F0ECFA002010BD10B50421002313
:102CD000C0F8F4111A46194600F0E1FA002010BDC0
:102CE00010B50A46024903A000F0E3F8004810BD01
:102CF00088050020437573746F6D20484944204354
:102D00006F6E6669670000001220088000487047F7
:102D1000FC00002010B50A46024903A000F0C9F8E3
:102D2000004810BD88050020437573746F6D2048FE
:102D3000494420496E746572666163650000000055
:102D40000420088000487047F800002010B50A46AB
:102D5000024903A000F0ADF8004810BD880500202E
:102D6000476175737300000010B50A46024903A05D
:102D700000F09FF8004810BD88050020476175737A
:102D80007320437573746F6D2048756D616E206993
:102D90006E746572666163650000000010B50A46D6
:102DA000024903A000F085F8004810BD8805002006
:102DB00030303030303030303030314100000000C1
:102DC000F8B5044648880D46010A082954D2DFE8C0
:102DD00001F05304091753534951D4F81012207CC1
:102DE0000A6819E0207C02260028D4F8140205D0D5
:102DF000C16A68468847014646704AE0816AF8E73A
:102E0000C1B2062926D2DFE801F0030A0F14191E09
:102E1000D4F81012207C4A686946904718E0D4F82C
:102E20001012207C8A68F7E7D4F81012207CCA6858
:102E3000F2E7D4F81012207C0A69EDE7D4F81012FA
:102E4000207C4A69E8E7D4F81012207C8A69E3E71D
:102E500001461EE0C1B2D4F814026A46836B2046D4
:102E60009847F5E7207C38B9D4F81402416B6846DE
:102E70008847EDE7207C20B129462046FFF7F3FE86
:102E8000F8BDD4F81402016B684688470146072054
:102E90004870BDF800000028F2D0EA88002AEFD080
:102EA000824200D90246ADF800202046FFF700FF1D
:102EB000F8BD70B5002300281DD00446002502E0AF
:102EC0006D1CEDB2641C2678002EF9D1022404EBAF
:102ED00045041480CC545B1C0322CA5400245B1CA0
:102EE00006E0CA545B1CDAB28C54521CD3B2401CAC
:102EF0000278002AF5D170BD10B580B1D0F8143237
:102F000013B10023C0F8143209B1C0F81012012126
:102F100080F8FC11027000F0AFF8002010BD022014
:102F200010BD10B50024D0F82002FDF795FC30B19B
:102F3000012801D0022801D0022400E0012420460B
:102F400010BD10B50024D0F82002FDF765FC30B1AB
:102F5000012801D0022801D0022400E001242046EB
:102F600010BD2DE9F0411746044641B1D4F81402D2
:102F700042698AB394F8FC01032842D043E0D4F8B4
:102F8000F411002504F11400022933D1D0E90263C1
:102F90009E4207D9F31A83609AB239462046FFF75A
:102FA0005AFE12E04068B0FBF3F103FB1101A1B936
:102FB000984212D3D4F8F81188420ED2002211465A
:102FC0002046FFF748FEC4F8F85100231A46194678
:102FD000204600F0BAF80DE012E0D4F81402C168FF
:102FE00029B194F8FC01032801D1204688472046E6
:102FF000FFF753FE94F80002012804D184F8005230
:1030000001E0204690470020BDE8F08170B51546EC
:10301000044641B1D4F8140282693AB394F8FC0131
:10302000032824D025E0D4F8F41104F58270032994
:103030001FD1D0E902218A420BD9531A8360084676
:10304000834200D303469AB229462046FFF7FBFD90
:103050000FE0D4F81402016929B194F8FC010328A7
:1030600001D1204688472046FFF72FFE01E0204689
:103070009047002070BD000010B51C490446C1F8FF
:103080001C04C0F820121A4808600820486002207A
:1030900088600320C86000208861C8610862084613
:1030A000FDF710FD20B140F2151112A000F0E4FD73
:1030B0000022D4F820021823114604F50874FDF705
:1030C00081FB5823002280212068FDF77BFB982399
:1030D000002281212068FDF775FBD8230022012101
:1030E0002068FDF76FFB002010BD00006801002084
:1030F000005C00402E2E2F5372632F757362645F45
:10310000636F6E662E6300000A06D0F8200201F09D
:103110007F0100EB411002D590F82A00704790F82B
:103120000A02704770B51D4613460024D0F82002ED
:103130002A46FDF7B5FB30B1012801D0022801D0A5
:10314000022400E00124204670BD10B50024D0F810
:103150002002FDF7C7FB30B1012801D0022801D0C1
:10316000022400E00124204610BD70B50022044670
:1031700040231146FFF7D6FF40252B460022802131
:103180002046C4F81051FFF7CDFF0120256284F8D6
:10319000FC01D4F8180228B1D4F81402217942684D
:1031A00020469047002070BD90F8FD1180F8FC117A
:1031B0000020704710B590F8FC11032904D1D0F815
:1031C0001412C96901B18847002010BD01740020A4
:1031D000704710B50024D0F82002FDF706FD30B18D
:1031E000012801D0022801D0022400E00124204659
:1031F00010BD70B5044600F50270054600F05FF89A
:103200000120C4F8F401B4F80E02C4F8F80194F8EF
:10321000080210F01F010AD001290DD0022910D098
:1032200000F08001204600F011F8002070BD294612
:10323000204600F0AAF8F8E72946204600F08CF96D
:10324000F3E72946204600F019F9EEE710B500240F
:10325000D0F82002FDF766FB30B1012801D002282A
:1032600001D0022400E00124204610BD10B5002446
:10327000D0F82002FDF7D4FC30B1012801D002289B
:1032800001D0022400E00124204610BD90F8FC117A
:1032900080F8FD11042180F8FC110020704710B562
:1032A0000024D0F82002FDF768FB30B1012801D0DE
:1032B000022801D0022400E00124204610BD0A7833
:1032C00002704A7842708A78CB7802EB03224280FF
:1032D0000A794B7902EB032282808A79C97902EB61
:1032E0000121C18070470246002011B1C2F81412BA
:1032F00070470220704710B5D0F8142202241AB18A
:103300001268904700B90024204610BD70B50E46E3
:103310001A4D897804462970032928D894F8FC01AD
:10332000022802D0032822D105E099B10320616070
:1033300084F8FC0109E091B1606888420AD0C1B20A
:103340002046FFF779FC297861602046FFF7D3FF1C
:1033500002280CD02046BDE87040FFF7B6BC022022
:1033600084F8FC0120466160FFF766FCF2E7314615
:103370002046BDE87040FFF776BC00000800002042
:1033800010B5FFF773FF002010BD2DE9F0410026B6
:103390004B78012532460A2B43D2DFE803F03C5834
:1033A0004251420805422A27FFF70AFD63E004461E
:1033B0008888C8B9C888B8B9887800F07F0794F8B9
:1033C000FC01032810D084F8FE7139462046FFF72F
:1033D00000FF2046FFF779FC1FB1022084F8FC01B2
:1033E00049E084F8FC5146E020461AE0FFF78EFFE2
:1033F00041E0CB88012B14D190F8FC31022B02D094
:10340000032B0ED104E08260012200F1080114E0D8
:103410000122011D11E090F8FC21022A04D0032AA8
:1034200002D0FFF720FC26E0C560D0F8041209B1F5
:103430000321C160022200F10C01FFF739FC1AE000
:1034400004464888012816D1C4F804520BE004460B
:1034500090F8FC01022801D00328C5D14888012832
:1034600009D1C4F80422D4F8140282682046904797
:103470002046FFF72AFC3046BDE8F08170B50D46C6
:103480000446287800260979C0F34110012806D0A7
:103490006878A0B301281FD003283FD107E0D4F8F3
:1034A00014022946826820469047002070BD94F897
:1034B000FC01022817D003282CD1688828B921B133
:1034C000802902D02046FFF7C1FED4F81402294615
:1034D00082682046904713E094F8FC01022802D04D
:1034E000032817D103E0C9B180291BD116E06888F1
:1034F000A0B9480604D02046FFF713FDE5E703E036
:103500002046FFF7E2FB09E094F8FC01022807D00F
:1035100003280BD029462046FFF7A5FB304670BD97
:103520004806FBD02046FFF791FEF7E7080601F0BA
:103530007F0004EB001501D5143501E005F5827517
:103540002046FFF7E1FD00B1012028600222294654
:103550002046FFF7ADFBE1E770B5054690F8FC01AA
:103560000C4603280DD1207903280AD8D5F8140277
:10357000826828469047E08830B92846FFF7A5FBC7
:1035800002E02846FFF76FFB002070BD7047000087
:1035900000487047480100202DE9F047CC780A78B0
:1035A00048F68F1334B1012C6DD0022C08D0032CB7
:1035B00013D10BE030F822401C4044F400730AE0C1
:1035C00030F822401C4020F8224006E030F822402B
:1035D0001C4044F4C06320F822300C7830F82450AA
:1035E00048F68F72154048F280031D43254320F8AA
:1035F00024508D7A48F6BF7904274BF68F7A48F22B
:10360000C0044CF28006EDB30D7830F825C048F2C6
:1036100080180CEA020C4CEA080C20F825C0CD8872
:10362000B0F850C025F0010591F800800CEBC80CF3
:1036300000EB4C0CCCF800540D89B0F850C025F0CC
:10364000010591F8008007EBC807674400EB4707C6
:10365000C7F800544D78002D0D7830F825704FEAEA
:1036600047477DD0002F05DA30F8257017403743E3
:1036700020F825700D7830F825707F0608D530F8D1
:10368000257001E024E01DE01740274320F8257055
:103690000C7830F824501540354320F824500C782D
:1036A00030F8242002EA09021A4320F824200A787C
:1036B00030F8221001EA0A01194320F822100020F4
:1036C000BDE8F08730F822401C4044F4806382E774
:1036D0004D78F5B18D88B0F8506025F001050F7870
:1036E00006EBC70600EB4606C6F800540D7830F826
:1036F0002560760605D530F825601640264320F86B
:1037000025600A7830F8221001EA090181F02001D1
:10371000D2E78C88B0F8505024F0010491F800C032
:1037200007EBCC073D4400EB4505C5F80044B0F875
:1037300050400D78062707EBC5052C4400EB4407E5
:103740000C694FF6FF7C07F580673E2C0CD9C4F35B
:103750004F15E40601D16D1EADB20CEA852400E0E0
:103760001EE044F4004407E0C4F34F05E40701D031
:103770006D1CADB20CEA85243C600C7830F8245006
:103780006D0405D530F824501540354320F82450F9
:103790000A7830F8221001EA0A0181F440518BE7DF
:1037A000002F05DA30F825701740374320F82570D0
:1037B0000D7830F82560760605D530F8256016407E
:1037C000264320F825600E7830F826501540254312
:1037D00020F826500C7830F8242002EA0A0282F4FD
:1037E00040521A4320F824200A7830F8221001EAC7
:1037F000090161E7002070472DE9F04391F80A8044
:1038000091F801C00A7848F6BF774BF68F7948F2F5
:10381000800348F2C0054CF2800648F68F74B8F178
:10382000000F2ED0BCF1000F30F822C04FEA4C4CF4
:103830004ED0BCF1000F07DA30F822C00CEA040CBD
:103840004CEA060C20F822C00A7830F822C05FEA61
:103850004C6C07D530F822C00CEA040C4CEA050C7D
:1038600020F822C00A7830F822502540354320F84D
:1038700022500C7830F824203A401A4320F82420B3
:103880001BE0BCF1000F0ED030F82260760605D5A3
:1038900030F8226026402E4320F822600A7830F863
:1038A000221039400EE030F822506D0405D530F872
:1038B00022502540354320F822500A7830F8221053
:1038C00001EA0901194320F822100020BDE8F08325
:1038D000BCF1000F07DA30F822C00CEA040C4CEA05
:1038E000060C20F822C00A7830F82260760605D54A
:1038F00030F8226026402E4320F822600E7830F8FF
:10390000262022402A4320F826200C7830F8242054
:1039100002EA09021A4320F82420BFE7002070477A
:1039200000207047012120F8401F00210180818084
:1039300001820846704730F8401F21F43D41018064
:10394000002070470020704730B54D780A78002D70
:1039500048F68F7430F8225048F2800312D06D067A
:1039600007D530F82250254048F2C004254320F8FE
:1039700022500A7830F8221048F6BF74214081F0B6
:10398000300111E06D0407D530F8225025404CF28B
:103990008004254320F822500A7830F822104BF694
:1039A0008F74214081F44051194320F822100020E7
:1039B00030BD10B50A7848F2800352B14978002929
:1039C00030F8221010D048F6BF74214081F0100169
:1039D0000FE001884BF6BF72114081F4805181F0F5
:1039E00010011943018007E04BF68F74214081F4E8
:1039F0008051194320F82210002010BD2DE9F0411C
:103A00000D460646896995F801C00023AA7A022767
:103A100028690C4648F28008BCF1010F05D08142AC
:103A200052D90446081AA8614FE0814203D90446DE
:103A3000081AA86100E0AB617AB1287836F8201046
:103A40004906B6F8501007EBC000084406EB4000EA
:103A5000C0F8004412D52A8911E0A3B2AA883046E2
:103A6000696900F0CEF8B6F85000297807EBC1017B
:103A7000084406EB4000C0F800441CE0EA88A3B20A
:103A80003046696900F0BDF8687848F68F7110B16A
:103A9000012807D00FE0287836F820200A4048F2A5
:103AA000C00105E0287836F820200A404CF2800159
:103AB0000A4326F82020297836F8210048F6BF72FC
:103AC000104080F0300067E0AB6106234FF6FF70D6
:103AD0001AB1BCF1000F1BD056E0B6F850102A788E
:103AE0003E2C03EBC202114406EB410202F5806258
:103AF00039D9C4F34F11E30632D000BF00EA812068
:103B000040F4004002E000BF00EA812010603BE08A
:103B1000B6F850102A783E2C07EBC202114406EB8F
:103B2000410202F580620BD9C4F34F115FEAC46C05
:103B300001D1491E89B200EA812141F4004108E027
:103B4000C4F34F015FEAC47C01D0491C89B200EA8A
:103B50008121116069780029BFD001290AD013E0C2
:103B6000491E89B2CAE7C4F34F01E307CCD0491C10
:103B700089B2C9E7B6F85000297807EBC1010844BB
:103B800006EB4000C0F80044297836F821004BF6D7
:103B90008F72104080F4405040EA080026F821005F
:103BA0000020BDE8F08130F8401F41F43D41018024
:103BB000002070470148FCF7FFBE000068010020AC
:103BC0000148FCF7F9BE000068010020B0F844008D
:103BD000704700005B1C00EB42005B0800F5806052
:103BE00006D000BF30F8042B21F8022B5B1EF9D160
:103BF00070470020704711B98021A0F84C100020B8
:103C0000704710B55B1C00EB42005B0800F580605C
:103C100009D011F8012B5B1E11F8014B42EA042276
:103C200020F8042BF5D110BDFEE7000033B57E214E
:103C300081B001EA40000E4D8DF800004FF4805431
:103C4000002221462846FCF7F8FC6423012269463D
:103C50000848FDF787FE6423012202A90548FDF705
:103C600081FE012221462846FCF7E7FC3EBD00000C
:103C7000000C014088070020FEE702E008C8121F80
:103C800008C1002AFAD170477047002001E001C145
:103C9000121F002AFBD17047FCF7E2FCFEF739FD4A
:103CA000FEF714FAFEF7A2FAFEF780FABD48BC4907
:103CB0004FF0000901604FF4E131C0E901190C2215
:103CC000C0F80C90C0E90492C0F81890C0F81C909D
:103CD000FEF7D7F800B1FEE70822B349B348FEF774
:103CE0003CFFB14C0A3CA070FEF761FC00224FF48F
:103CF0000051AF48FCF7A1FC00F060F9DFF8B4B266
:103D00004FF480715846FCF793FC30B1FCF7A0FBF0
:103D1000A948FCF74FFAFCF75DFBFCF76BFAA246EB
:103D2000A04CA14D5A346D1F9E4926204A31FEF702
:103D30002FF956468AF8040008BB9A484A30FEF725
:103D400006F93071D8B99748283050F8221FC6F8C4
:103D500005100079707200F03BF9E07B08B1FF2894
:103D60000DD12878207068786070A878A070E87805
:103D7000E070287920710120E073FCF773FAE17B91
:103D8000481E022861D2307801285ED17078401C2C
:103D900070702878F0B3227890424FD06A78CAB316
:103DA00063789A424AD0AB78A3B3A778BB4245D098
:103DB000EF787FB394F803C067453FD095F804804F
:103DC000B8F1000F3AD094F804C0E04536D094F82A
:103DD00005C0604532D094F806C062452ED094F8F4
:103DE00007C063452AD094F808C0674526D094F8E8
:103DF00009C0E04522D002290BD1A072E2722373E0
:103E0000677384F80E800320E073FCF72BFA86F8C2
:103E1000009000E012E0E07B01280FD1287860716B
:103E20006878A071A878E071E878207228796072CB
:103E30000220E073FCF716FA86F800907078C82824
:103E400003D986F8019086F800900C20FCF732FA2E
:103E5000E07B00283FF468AFFF28FBD028780028DB
:103E6000F8D068780028F5D0A8780028F2D0E87853
:103E70000028EFD028790028ECD04FF4007739469D
:103E8000D8465846FCF7D4FB30BB287821788842C6
:103E900022D16878617888421ED1A878A1788842BA
:103EA0001AD1E878E178884216D1287921798842B8
:103EB00012D1012251033E48FCF7BFFBFA20FCF768
:103EC000F9F9002239013A48FCF7B7FB4FF4FA70D0
:103ED000FCF7F0F901203070394646464046FCF7C1
:103EE000A7FB30BB28786179884222D16878A17914
:103EF00088421ED1A878E17988421AD1E878217ADF
:103F0000884216D12879617A884212D14FF400583C
:103F1000012241462648FCF790FBFA20FCF7CAF93B
:103F2000002241462248FCF788FB4FF4FA70FCF768
:103F3000C1F939463046FCF77BFB30BB2878A17AC3
:103F4000884222D16878E17A88421ED1A878217B04
:103F500088421AD1E878617B884216D12879A17B02
:103F6000884212D10122124F560331463846FCF7DF
:103F700064FBFA20FCF79EF9002231463846FCF734
:103F80005CFB4FF4FA70FCF795F985F8009085F822
:103F9000019085F8029085F8039085F80490C3E6B7
:103FA00000380140E0070020180100204C080020E4
:103FB00000100140000C014000FC000810B5372043
:103FC000FEF714FB0149C87010BD00000E0100206F
:103FD0002DE9F0414A4C0120002520702720A070D7
:103FE000E57025716571A571E57108222146454886
:103FF000FEF7B3FDA4F10A07B8708220FCF75AF966
:104000002570A570E57025716571A571E5710822AF
:1040100021463C48FEF7A1FDB8708220FCF74AF922
:10402000661F3078000900F06FF8A070307800F05B
:104030000F0000F069F8E0707078000900F064F893
:104040002071707800F00F0000F05EF86071B078B9
:10405000000900F059F8A071B07800F00F0000F0EE
:1040600053F8E071082221462648FEF776FDB87025
:104070008220FCF71FF92570A570E5702571657128
:10408000A571E571082221461E48FEF766FDB8704D
:104090008220FCF70FF9F078000900F035F8A070E5
:1040A000F07800F00F0000F02FF8E0703079000990
:1040B00000F02AF82071307900F00F0000F024F8A9
:1040C00060712820A071E571082221460D48FEF795
:1040D00044FDB8708220FCF7EDF82570A570E570FE
:1040E00025716571A571E571082221460548FEF725
:1040F00034FDB870BDE8F0418220FCF7DBB8000069
:10410000180100204C080020010021D0012922D0F4
:10411000022923D0032924D0042925D0052926D01B
:10412000062927D0072928D0082929D009292AD0EB
:104130000A292BD00B292CD00C292DD00D292ED0BB
:104140000E292FD00F2830D001D94FF038007047FA
:104150004FF0270070474FF01E0070474FF01F00D0
:1041600070474FF0200070474FF0210070474FF02C
:10417000220070474FF0230070474FF02400704733
:104180004FF0250070474FF0260070474FF00400B5
:1041900070474FF0050070474FF0060070474FF032
:1041A000070070474FF0080070474FF00900704754
:1041B00000000000000000000102030406070809D7
:1041C0000000000001020304E84100080000002094
:1041D000240100007A3C00080C4300082401002060
:1041E0004C0D00008A3C00080000000000000000A8
:1041F00000000000012B0008952A0008812B000810
:1042000000000000C72A0008652A0008712A00087B
:10421000000000000000000000000000E92A000883
:10422000E92A0008E92A0008F52A00080000000031
:1042300009022900010100C0320904000002030044
:104240000000092111010001223F0007058103023E
:1042500000200705010302002000000009211101D0
:104260000001223F000000000A060002000000409A
:104270000100000005010906A101050719E029E771
:1042800015002501750195088102950175088103C6
:104290009505750105081901290591029501750318
:1042A0009103950675081500256505071900296510
:1042B0008100C0008C0000208D01000889010008E9
:1042C00091010008092D0008412D00084D2D00081E
:1042D000692D00089D2D0008E12C0008152D00080F
:1042E0000403090412010002000000408304505737
:1042F00000020102030300000000000000000000B3
:0C430000000000000000000000A24A04C1
:04000005080000ED02
:00000001FF
